:030000000219FDE5
:03000B000200A848
:03002B000201547B
:03005B000202D4CA
:030073000202C1C5
:1000800002030406080C10182030406080040608A3
:100090000C10182030406080A0C00003070F1F051F
:1000A000050D050205030302C2AFC0D0C0E0206207
:1000B00014E5256009E473E525F4F58AD262D0E001
:1000C000D0D0D2AF3285268AC262E526F46029D02C
:1000D000E0D0D0C292C291C290D2AF32C292C2914D
:1000E000C290206F0C2065097405D5E0FDE57B42C8
:1000F00090D0E0D0D0D2AF32758A00C28DD26201EA
:10010000F101B7306805206502D29201B730680569
:10011000206502D29101B7306805206502D29001B6
:10012000B7C29530680A2065077446D5E0FDD292C3
:1001300001B7C29430680A2065077446D5E0FDD245
:100140009101B7C29330680A2065077446D5E0FD77
:10015000D29001B7C2AFC2AD53E6EFC0D0C0E0D27B
:10016000D3D2AFC2CEE52A6007207449152A21B543
:100170007800790020742EE580307E01F430E702AB
:1001800078FF53DACF207E0343DA20307E0343DA50
:1001900010C2D8C271E580307E01F430E70279FFE9
:1001A000C3E89970CB306103752A18207403752A4F
:1001B00018885CD27020740DE52B6004152B21C5C6
:1001C00043DA01C2D82070024138A85C206102C223
:1001D00070207431C3E894F0400374F0F8E8C4541C
:1001E0000F28F87984B703024105C313C31387218D
:1001F000200802C313200A06C3C898F8410528F84E
:10020000500374FFF8C3E895655003E565F888224C
:10021000E52D54066022206B1FE536C333C333F847
:10022000E564C313C313F9C3952240028922E8256C
:1002300022F52250037522FF852224A824C3E52439
:1002400095614002A8618825E5667002417CC3E89B
:10025000AA669A5003E8FAE4F9EAC333FBE568F4C6
:100260005B29400D2567F8E56760021567400B4183
:100270007C0AC3E5679A5002056778FF882620CF7D
:100280000AD0E0D0D043E610D2AD32C2CF053A78E2
:1002900001E52A6005307402152AC3E55C9401402B
:1002A00005755F0041B7756000756900E55F240161
:1002B000F55F5003755FFFD0E0D0D043E610D2ADBC
:1002C00032C2AF53E67F7592FA7593FFC2607591A3
:1002D00004D2AF32C2AF53E6EFC2ADC0D0C0E0C06F
:1002E000F0D2D3D2AFA8FBA9FCC2D8307102613BD7
:1002F00053DACF207E0343DA10307E0343DA20D274
:1003000071E580307E01F420E70261128827892898
:10031000A16853DACF207E0343DA20307E0343DA2C
:1003200010C2D8C271307402A1547800E580307ECA
:1003300001F430E702A154885CA13C53DACF207E5F
:100340000343DA20307E0343DA10C2712061028158
:100350001453DACF207E0343DA10307E0343DA20D1
:10036000C2D8D27188578958C3E89555F8E995568F
:10037000F97B007E087A00C3E8948CE9940050056C
:10038000755B008106882178A2E6A8216055C3E844
:1003900094C8E994005008E4D2E4FB7A0A61E1C30E
:1003A000E89468E994015008E4D2E3FB7A0F61E134
:1003B000C3E894D0E994025008E4D2E2FB7A1E61CB
:1003C000E1C3E894A0E994055008E4D2E1FB7A3C4B
:1003D00061E1C3E89498E994085008E4D2E0FB7A1C
:1003E000787E00C3E89559FCE9955AFD30E70AECA0
:1003F000F42401FCEDF43400FD755B00C3EC9AEDD0
:100400009E5003755B018859895A85575585585602
:100410007802A13CC3E89527F8E99528F9307C02D9
:10042000A120307B02A120307A02A119207502811F
:1004300037E9FDE8FC8156E9C313F9E813F8307990
:1004400002A119E9C313F9E813F8307802A119E9F8
:10045000C313FDE813FC20612CC3EC941CED940243
:100460004002816DED701EC3EC94C850180529E55B
:0E0470002970021529C3E529940A5002A154EF
:10047E00755C00D270A154E529600215297888E6D2
:10048E00F97400207F087896B90302789EE624FA64
:10049E00FEE43400FFC3EC9EFCED9FFD9208B90311
:1004AE0010A2085007207609D27681BF307602C29C
:1004BE0076A2085016B9030DECF42401FCEDF434C9
:1004CE0000FD0204D978007900A120B90315EC33A0
:1004DE00FCED33FDC3EC940AFCED9400FD50047C5E
:1004EE00007D00C3EC94FFED9400400678FF790088
:1004FE00A120EC8572F0A4C5F0A2F733F879004084
:10050E000302053C78FF790002053CE9C313F9E8C4
:10051E0013F8307C0EE9600278FFC3E81338F8E474
:10052E003400F9C3E894FFE99400400278FF885C38
:10053E00D270206102A154741FF4552F4BF52FC2B7
:10054E0074EB7002D274752A18307403752A0A304F
:10055E006102A16820740353DAFE207403752B0622
:10056E00D0F0D0E0D0D0D2AD43E610327901020502
:10057E00987903020598790A020598791E02059862
:10058E00796402059879C80205987817E4D5E0FDDC
:10059E00D8FAD9F6227A147B780205BF7A107B8CB2
:1005AE000205BF7A0D7BB40205BF7A0B7BC802052C
:1005BE00BFE573D5E001227902E4C294D5E0FDD205
:1005CE0091D5E0FDC291D5E0FDD294D5E0FDE920B4
:1005DE00E002D29230E002D290E573D5E0FDE92040
:1005EE00E002C29230E002C2907496D5E0FDD9C905
:1005FE00EAF8D5E0FDD8FBDBB8C29422C37C007DBF
:10060E000075F00005F0EA33FAEB33FB50F6EB130E
:10061E00FBEA13FAC3E9FFE8FEE89AF8E99BF95002
:10062E0004EFF9EEF8B3EC33FCED33FDD5F0DFED6E
:10063E00F9ECF822E889F08A20D2D4F8A9F07B00F0
:10064E0030F70B7BFFF42401F8E9F43400F9E88568
:10065E0020F0A4ADF0F8E98520F0A4AFF0FEED2E69
:10066E00F974003FFA7C04C3EA13FAE913F9E813AC
:10067E00F8DCF48BF030F70AE8F42401F8E9F434EE
:10068E0000F9E889F0C2D4F8A9F02222C3E541139B
:10069E00F9E54013F8C3E54498F8E54599F9500C8F
:1006AE00C3E89480E994FF40160206D1C3E8947F14
:1006BE00E9940050030206D1787F79000206D178C2
:1006CE008079FF8849894A22E5492546F8E54A3569
:1006DE0047F9854A20E4300701F43548FA30E70936
:1006EE00C3EA94F0401502070FC3EA940F500302B9
:1006FE00070F78FF79FF7A0F02070F780079007ADB
:10070E00F0C3E5249561500AC374019524500B0281
:10071E00072DE54A20E70E02072DE54A30E7068849
:10072E004689478A482278A5E6FAC3E54933F8E5B3
:10073E004A33F9D142E930E70BC3E89480E994FFDC
:10074E004013E167C3E8947FE994005002E16778B3
:10075E007F7900E167788079FFE820E715C3E5230C
:10076E0098F84009C3E89401400302078E7801020D
:10077E00078EE8F424012523F8400302078E78FF44
:10078E00884B2278A6E6FAA847A948D142E930E775
:10079E000CC3E89401E994FF40160207C2C3E89423
:1007AE00FFE9940050030207C278FF79000207C2E6
:1007BE00780179FFE920E715C3E54B98F84009C3A6
:1007CE00E8940140030207E978010207E9E8F424FE
:1007DE0001254BF840030207E978FF88242278FFB1
:1007EE0020692879A1E76023E541601F74FF8541E8
:1007FE00F0848539F0306A0375F005A4F8C5F06011
:10080E000278FFC3E895645002A864886322C3E5AA
:10081E00409440E5419401E563500314012D0460BA
:10082E0002F563220208352275E890227883E6FFEE
:10083E0030EDF9A8BDA9BE0570C3E570940840520D
:10084E00757000E9FA79A0E76044EA7007E5716017
:10085E001B02086EC3E895716010E5715006600CBE
:0F086E001402087A0460F902087AE571F571C383
:10087D00946D401B7561C0C394044013756180C3B2
:10088D009404400B756140C3940440037561007579
:10089D00BB0622E561F460020561E570B4070375DE
:1008AD00BB1022743279A787F0A4C5F0A2F733F8F4
:1008BD00C3E895614002A86188228824882588268E
:1008CD008864227540007541F022C2AF75C820A81A
:1008DD00CCA9CDAA3A30CF010A75C824D2AFAB3B13
:1008ED00AC3C883B893CC3E89BF8E99C206908F93E
:1008FD0030660221E62140AD3D8A3DF9EA9DFA6060
:10090D000478FF79FFAE3EAF3F8B3E8C3FA83BA9ED
:10091D003CC3E89EF8E99FF9C3E54113FBE540139D
:10092D00FAE82AF540E93BF54150067540FF75415F
:10093D00FF218DAA40AB41AC40AD417E047F02C387
:10094D00EB9404400D1E1FC3EB94084005206A0272
:10095D001E1FC3ED13FDEC13FCDEF7C3EA9CFAEB8F
:10096D009DFBEF6009C3E913F9E813F8DFF7EA28F7
:10097D00FAEB39FB8A408B4150067BFF8B408B4154
:10098D00C3EB94025002D2663069047F0321B8781C
:10099D0092E6FFC3E537948240110FC3E53794A06B
:1009AD0040010FC3EF940640027F057E02E541C46E
:1009BD00540FF9E541C454F0F8E540C4540F28F83C
:1009CD00C3E89EFAE99400FB4009C3EA9402EB9454
:1009DD000050047A02E4FB4132AA40AB41EBC4FE65
:1009ED00EAC4540F4EFCC3EA9CFAEB9400FBC3E837
:1009FD0013C313F8EA28FAEB3400FB8A408B41C38A
:100A0D00EB94024002C2667802EBC4FE7B00EAC49E
:100A1D00540F4EFAC3EA98FA4005C3940250027A75
:100A2D00027892E6FF3060024132855192855293F1
:100A3D00D26043E680C3E49AF8E49BF93066024144
:100A4D00BEE8FAE9FBD3E913FDE813FC885189529E
:100A5D00C3EF94036038EF20E00DE82CF8E93DF981
:100A6D00ECFAEDFB020A87E828F8E939F9C3E82426
:100A7D0002F8E93400F97AFE7BFFC3EF9403400ED0
:100A8D008A538B54884D894E8C4F8D5041F288532B
:100A9D0089548A4D8B4E8C4F8D503069127553F0A1
:100AAD007554FF754FF07550FF7551F07552FF413C
:100ABD00F2E8FAD3E813FC8851C3EF94036020EFFA
:100ACD0020E007E82CF8ECFA41DEE8282402F87A59
:100ADD00FEC3EF940340088A53884D8C4F41F28832
:100AED00538A4D8C4FE568C3335002646BF5683003
:100AFD00600241FC753402D26043E680E52D540658
:100B0D006034A840A941C3E913F9E813F8C3E91308
:100B1D00F9E813F8306904E92440F9C2AF53E67FD0
:100B2D00759100C3E498F594E499F595759104D207
:100B3D006043E680D2AF22D2647543007520003049
:100B4D006C03752040020B63D26475430075204021
:100B5D00306C0375200078017901206620E52D5455
:100B6D00066002C2647914E541C313700104F8C331
:100B7D00941440027814306904781B791B2060109E
:100B8D00E543600C306903D53404D26D810E7104D8
:100B9D000543E59BF45440B5200261F8306909081E
:100BAD00C3E899400118618A20640A08C3E8994096
:100BBD00026163618AC264C2AF53E67F75910030F2
:100BCD0066127594007595F8759104D26043E680B0
:100BDD00D2AF6163E5417EFFC3334005C3334001AE
:100BED00FEC3E49E759400F59561D5C3E53394017C
:100BFD00500261633064026163D802810C618AC264
:100C0D006DC2AF53E67F75910085539485549575EC
:100C1D009104854D92854E93D26043E680D2AFE527
:100C2D002D54066008206A020533020C4A306D0D02
:100C3D00206C0A20640715811581021507227800A2
:100C4D003064027801E53775F007A4F9E5F028F571
:100C5D00F0E9A2F013A2F113A2F213F537C39478C1
:0E0C6D005003753778C3E53795384008D265D7
:100C7B00C292C291C2903060028181854F928550A1
:100C8B0093D26043E68022207D16C2AF754202C22A
:100C9B0094D295306202D290D2AF759F11020E8121
:100CAB00C2AF754202C294D293306202D292D2AFDB
:100CBB00759F11020E81307243207D20C2AF7542A9
:100CCB0003900132757B10C290C293306204D291B3
:100CDB0081DFD294D2AF759F01020E81C2AF7542F4
:100CEB0003900132757B10C292C295306204D2918F
:100CFB0081FFD294D2AF759F21020E81207D17C246
:100D0B00AF75420390010DC290306202D291D2AF07
:100D1B00759F01020E81C2AF75420390010DC29205
:100D2B00306202D291D2AF759F21020E81207D16C7
:100D3B00C2AF754204C295D293306202D291D2AF48
:100D4B00759F21020E81C2AF754204C293D29530BA
:100D5B006202D291D2AF759F01020E813072432095
:100D6B007D20C2AF754205900121757B20C291C2D7
:100D7B0094306204D292A185D295D2AF759F1102A5
:100D8B000E81C2AF754205900143757B08C291C2BB
:100D9B0094306204D290A1A5D293D2AF759F110269
:100DAB000E81207D17C2AF754205900103C29130B1
:100DBB006202D292D2AF759F11020E81C2AF754201
:100DCB0005900117C2913062EBD290D2AF759F1193
:100DDB00020E81207D16C2AF754206C293D29430AB
:100DEB006202D292D2AF759F01020E81C2AF7542E1
:100DFB0006C295D294306202D290D2AF759F210277
:100E0B000E81307243207D20C2AF754201900143A9
:100E1B00757B08C292C295306204D290C12BD293DB
:100E2B00D2AF759F21020E81C2AF75420190012195
:100E3B00757B20C290C293306204D292C14BD29583
:100E4B00D2AF759F01020E81207D17C2AF75420193
:100E5B00900117C292306202D290D2AF759F2102DD
:100E6B000E81C2AF754201900103C290306202D273
:100E7B0092D2AF759F01C26522900101757B00C2B2
:100E8B0092C291C290C295C294C293C262227880E0
:100E9B0076FF0876FF0876FF0876FF08760308765C
:100EAB000408760B087601087601087601788C76B3
:100EBB00010876FF0876FF0876FF0876FF0876FFB5
:100ECB000876030876FF0876FF0876FF0876250874
:100EDB0076D00876FA0876FA0876040876FF087654
:100EEB000108760008767A0876FF08760108760105
:100EFB00087600087603087600227887E6FFC27230
:100F0B007888E6C394036008C27DE630E102D27DA7
:100F1B00C27E7889E630E102D27EC3EF940260088C
:100F2B00758E01D273020F38758E00C273227880D2
:100F3B00E6149000809378A5F67881E614900080F3
:100F4B009378A6F67886E61490008D9378A7F678BA
:100F5B0086E6F539C394025003753902789CE67521
:100F6B0038FFB402037538A0B4030375388278A335
:100F7B00E61490009A93F566D18422227896E6FACD
:100F8B007897E6FB7888E6B40305C3EB940EFB3049
:100F9B007F047A007BFFC3EB9AFCC3948250027CE4
:100FAB00827572000572EC8572F0A4C3E5F0947D36
:100FBB0040F222D27FF1871205891205897A007BD4
:100FCB00007C1012057FE55C2AFA74003BFBDCF316
:100FDB007C04C3EB13FBEA13FADCF7FEC27FF18749
:100FEB0022757C00757D00E5EF20E603752000057A
:100FFB0020903FFFE520146006901DFF14600093C6
:10100B0004600375EF1453D9BF7581C043FF801281
:10101B00057A75EF0443B203E5B3240220E70DF51F
:10102B0021E5E320E0068521B343E301120E84752D
:10103B0080FF75A40075F19075D47F75900075A530
:10104B003F75F23F75D50075A60175E241120E840E
:10105B00E4F8F6D8FD756801120E991215587898B8
:0D106B008673753001C2AF1205931205A304
:101078001205891205AA1205891205B112058912ED
:10108800167512059312059312058EC2AF757C0072
:10109800757D0078FA79FA308707D9FBD8F7021CF2
:1010A80000120F05120F39120F86120F87789886D3
:1010B80073120E8475881075890275C82475910499
:1010C80075D84075A82275B80275E690759B80752D
:1010D8009D0075D10E75BC5875BB0675BA1175E8BB
:1010E8008012057AD2AF12083275360053DACF2053
:1010F8007E0343DA20307E0343DA1043DA01C2D894
:10110800C271120593D2617B037A0CE55B70077A92
:101118000CDB03021093120589207003021093C29E
:1011280070E55CC3940240E1E52F541F855E5DF5D0
:101138005EB55DD5DAD5C26153DACF207E0343DAD6
:1011480020307E0343DA10C2D8C27178A2E6700854
:10115800D274E52F54E0F52FC27575290012058E5B
:10116800307409C3E529940A4002D27512057F78C4
:10117800023074027800C3E55C9840F0C2AF1205F3
:10118800A31205A31205A3D2AF120593754C0078DC
:1011980088E6B40302419312057F788CE6C3940174
:1011A8005003021293E530C3940150030212937561
:1011B8007CA5757DF1207435C3E55C94FF5003026E
:1011C8001293C2AF1205B8D2AF12058EC3E55C9474
:1011D8000150EFC2AF1205A31205841205A3D2AFC6
:1011E80012058EC3E55C94FF40E90216FA7F05D22A
:1011F8007F120F8712058EC2AFC27F120F87AE5CB7
:10120800C3E55C947FD2AF500241A312057AC2AF06
:101218001205B8D2AFDFD8120FBEC3EE9405789787
:10122800F612059312167D7F0AD27F120F871205D8
:101238008EC2AFC27F120F87AE5CC3E55C947FD2CB
:10124800AF50E412057AC2AF1205A3120584120545
:10125800A3D2AFDFD4120FBEEE24037896F6F87946
:1012680097E7C394824003985006E824827897F65B
:1012780012059312159A1216AC12058E120F87C317
:10128800E55C94FF500221B70216FA757C00757D63
:1012980000C3E55C954C4003855C4C12058E7801D3
:1012A8007988E7B403027805C3E55C984002219782
:1012B800C2AF1205B81205B81205B8D2AF1205931D
:1012C800753000E4F531F5320531E531F4703F054C
:1012D80032789AE67819146012783214600D787DA5
:1012E80014600878FA146003753200C3E532984038
:1012F8001D120E8412057A1532753100789986739D
:10130800C2AF1205B8D2AF7898867312058E12054F
:1013180084E52A70053074020193780120740278FC
:1013280006C3E55C9840A17888E6C394036003127D
:10133800058EE52A7003021093C2AF120E84E4F5FD
:1013480022F523F524F525F526F567D2AF7885E64D
:10135800C333F565E4F544F545F546F547F548F535
:1013680070F52CF52DF53775700875BB1012057AD8
:1013780012083630EDFDA8BDA9BEE97001F88871E4
:1013880012083A75700875BB10120F05C2AF756167
:10139800FF1208B0852261852262852263D2AF756B
:1013A8002201752401752501752601856069756A14
:1013B800017888E6B40307C27D307602D27DD26810
:1013C800D269753300120DDE120E0D1208D0120804
:1013D800D71208D01208D71208D0120B5512069946
:1013E800120C4B120C921208D7120B44306E0312D7
:1013F800069A2066031207EC30660312081C120CCA
:101408004B120CC11208D7120B55306E031206D6B8
:10141800120C4B120D381208D7120B44306E0312FF
:101428000734120C4B120D671208D7120B55306E89
:1014380003120791120C4B120DDE1208D712083650
:10144800120B44120C4B120E0D12083A1208D73028
:10145800692F856461856462856069756A01791898
:0E1468007A0CC3E53399400CC269D26A8A350A
:101476007561FF021489C3E55C940140030213E21F
:1014860002150F306A1D206C1AE535147006C26A03
:10149600D26B61E2F535C3E55C940140030213E2C9
:1014A60002150F753600788279A4E760027803C3C7
:1014B600E55F985054307404E52A604D7888E6B4A8
:1014C6000317207D0520760781DF30760281DF2035
:1014D6006C07D26C856461812178F0306C05856477
:1014E600617820C3E54198500261E2306C1BC26C02
:1014F600C27D307602D27DD26A753512856461610D
:10150600E20536E55C6002A112753600C2AF120E26
:10151600847887E6FE7602120F057887EEF6E4F504
:1015260022F523F524F525F526F565752C00752D90
:1015360000D2AF12058E120E8478A4E66006D2920F
:10154600D291D290307409C3E536940440020193D7
:1015560041CB901A0D78201215DCE520B45A0CA365
:101566001215DCE520B4A50302157A120E991215A0
:101576009A021599901A0378807B0A1215DCA30843
:10158600DBF9901A0F788C7B191215DCA308DBF9AE
:10159600901A2822C2AF12161F1215FC901A007458
:1015A6000E1215E1A374071215E1A374151215E1C5
:1015B600901A0378807B0A1215E0A308DBF9901ACB
:1015C6000F788C7B191215E0A308DBF9121632127C
:1015D6001610901A2822E493F622E6438F01538FC1
:1015E600FDFFC3E583941C400122EF857CB7857D12
:1015F600B7F0538FFE22438F02438F01857CB78558
:101606007DB7901A0DF0538FFC22901A0D745AB1C3
:10161600E1901A0E74A5B1E1227A3079D078209043
:101626001A40B1DCE520F709A3DAF7227A3079D03F
:10163600901A40E7B1E109A3DAF922AB74A875BBA9
:1016460001027984BB02027985BB03027986BB0459
:10165600027992BB05027987BB060279A3BB070212
:10166600799CBB08027988BB09027989E8F7227C54
:1016760005120593DCFB22C2AF1205A31205AA12BE
:1016860005B11205B81205841205A31205AA1205A2
:10169600B11205B81205841205A31205AA1205B1E6
:1016A6001205B8D2AF22C2AF1205B81205B11205A3
:1016B600AA1205A31205841205B81205B11205AACD
:1016C6001205A31205841205B81205B11205AA1255
:1016D60005A3D2AF22AE74AF75C2AF1205A3120531
:1016E600A31205A3120584DEF21205B8120584DFE3
:1016F600F8D2AF22D17DD175D1757574017575019A
:10170600757600D1DB7C05AD5C120593C3ED955C67
:1017160070F5C3E55C9401400AC3E55C94FF403272
:10172600021736D141B19AD17DC2AF75EF14D1758A
:10173600DCD50576C3E5769403500280C6D17505DF
:1017460075E5741490009F93F808C3E575985002E8
:1017560080AED175D1750574C3E574940A500280C4
:0D1766009C120E99B19AC2AF75EF14D175A7
:0319FD00020FECEA
:101A00000E0715FFFFFFFF03040B0101015AA5019B
:101A1000FFFFFFFFFF03FFFFFF25D0FAFA04FF01DE
:091A2000007AFF0101000300FF40
:101A400023585031324123202020202020202020E4
:101A500023424C48454C4923463333302320202031
:101A60002020202020202020202020202020202076
:101C0000C2AFC2D353D9BF7581C043B20343FF8073
:101C1000752438752503B1DC7529A5752AF175E29F
:101C20004043F18053A47F75D4FFD2877DFA7803B7
:101C300079E67C10752200752300901DE97B0675FE
:101C400024987525013087028145208708D8FBD963
:101C5000F9DCF781B7308708D8FBD9F9DCF781B711
:101C6000B19CE493A3C39A6004DDC381B7DBDBB10D
:101C70008E6002812E7B08E493FAA3B16FDBF87AC1
:101C800030B16F752200752300B18EEAFCEBFDC305
:101C9000ED94FE400EB18E8A278B28ED30E0048A49
:101CA000828B83B18E7AC270D8C3ED94FE601950D6
:101CB000CEBD002BEC600F7520007521FF7529004B
:101CC000752A000200008100A827A9280809D80465
:101CD000D90281DCB192EA89AAF281CE0D81A3C337
:101CE000ED94035053EDA2E092007AC5C3E58294CF
:101CF00000E583941C508A200010438F02438F011B
:101D00008529B7852AB7F0300029A827A92808090E
:101D1000438F01538FFDD804D902A133C3E58394C7
:101D20001C4003A3A11689AAE28529B7852AB7F02A
:101D3000A3A116538FFC817F7AC1BD030CE493A34A
:101D4000FAB153DCF8B14B817F8181AA22AB23B178
:101D50006FEBFAEA6222752608C3E52313F523E543
:101D60002213F52250066323A0632201D526EAB18F
:101D7000DCB1DC75260AEAF4200102D287300102C8
:101D8000C287B1DCC3134002C201D526EB22B19257
:101D9000EAFB208702A192308702A197752608AE40
:101DA00024AF25C3EF13FFEE13FEB1E0B1DCC3EAAD
:101DB000133087024480FA30E703632201C3E5232E
:101DC00013F523E52213F52250066323A0632201B5
:101DD000D526D9E52265236523F52222AE24AF2539
:101DE0000E0FDEFEDFFCD20122424C48656C6934E6
:071DF000373163F3300601F7
:00000001FF
